:020000040000FA
:020000009F2D32
:08000800FF000308FE000A08D6
:10001000FC000408FD008312031300308A00233023
:100020008100A10A063021020318A1012014A20FA9
:100030001C28A30F1C28A0143D08003E03193C28CF
:100040002E1C3A2883160313DB3086008312031319
:10005000860106155B230130652300001E30A400D5
:10006000061107306523061506306523A40B3028DA
:1000700006115E285B233E28502349231430A50037
:10008000FB01FA01EF21F521032254238501210808
:1000900003196920013021020319AA20023021022C
:1000A0000319EB200330210203192C210430210213
:1000B00003196D21053021020319AE210B118B1795
:1000C0007D0884007C088A007E088300FF0E7F0E76
:1000D0000900B830840001080002031C7A17B93007
:1000E000840001080002031CFA167A16BA30840054
:1000F00001080002031CFA15BB308400010800024D
:10010000031C7A15A330840001080002031CFB16AF
:10011000A230840001080002031C7B16FB15A130ED
:10012000840001080002031C7B15A0308400010834
:100130000002031CFB14831603137B0885007A0856
:100140008600831203138030860001308500A50BE2
:1001500069280800BC30840001080002031CFA175B
:10016000BD30840001080002031CFA16BE30840072
:1001700001080002031C7A16FA15BF30840001083A
:100180000002031C7A15A730840001080002031C3A
:10019000FB167B16A630840001080002031CFB1529
:1001A000A530840001080002031C7B15A4308400E4
:1001B00001080002031C7B14831603137B088500CF
:1001C0007A088600831203134030860002308500CF
:1001D000A50BAA280800C030840001080002031CF7
:1001E000FA17C130840001080002031C7A17C230DC
:1001F000840001080002031C7A16C3308400010841
:100200000002031CFA157A15FB16AB3084000108B6
:100210000002031C7B16AA30840001080002031CA4
:10022000FB15A930840001080002031CFB14A83050
:10023000840001080002031C7B14831603137B084F
:1002400085007A088600831203132030860004306C
:100250008500A50BEB280800FA17C43084000108BC
:100260000002031C7A17C530840001080002031C39
:10027000FA16C630840001080002031CFA15C730C4
:10028000840001080002031C7A15AF3084000108C5
:100290000002031CFB16AE30840001080002031CA0
:1002A0007B16AD30840001080002031C7B15AC30C6
:1002B000840001080002031CFB147B148316031343
:1002C0007B0885007A0886008312031310308600AD
:1002D00008308500A50B2C290800C83084000108CF
:1002E0000002031CFA177A17C930840001080002C3
:1002F000031CFA16CA30840001080002031C7A1697
:10030000CB30840001080002031C7A15B33084004E
:1003100001080002031CFB16B23084000108000231
:10032000031CFB15B130840001080002031C7B157F
:10033000FB14B030840001080002031C7B148316F8
:1003400003137B0885007A088600831203130830A4
:10035000860010308500A50B6D290800CC30840084
:1003600001080002031CFA17CD30840001080002C6
:10037000031C7A17FA16CE30840001080002031C11
:100380007A16CF30840001080002031CFA15B7303A
:10039000840001080002031C7B16B63084000108AB
:1003A0000002031CFB157B15B53084000108000218
:1003B000031CFB14B430840001080002031C7B14EE
:1003C000831603137B0885007A08860083120313C3
:1003D0000430860020308500A50BAE2908000310EC
:1003E000260DAF00FC21B20008000310260D013ECF
:1003F000AF00FC21B300080002308A002F08073E3E
:1004000003188A0A820032088A0033088200023404
:1004100047340234523402345A34023462340234DF
:100420006A340234723402347A3402348634023448
:100430008A340234963402349A340234A6340234B4
:10044000AA340234B6340234BA340234C634023424
:10045000CA340234D6340234DA340234E634023494
:10046000EA340234F6340234FA3403340634033402
:100470000A340334163403341A3403342634033470
:100480002A340334363403343A34033446342D10DA
:100490003030B10028184F2A0630A600482B013012
:1004A000A600482B2818572A0030A600482B0230F7
:1004B000A600482B28185F2A0030A600482B0330DE
:1004C000A600482B2818672A0430A600482B0330C2
:1004D000A600482B28186F2A0030A600482B0530AC
:1004E000A600482B2818772A0730A600482B003092
:1004F000A600482B2818842A003031070319822AC5
:10050000B10B482B2D14482BA601482B2808AC0012
:10051000A60A482B2C082806031D902AA601482B62
:1005200028182B10281C2B14A60A482B2808AC00CE
:10053000A60A482B2C082806031DA02AA601482B32
:1005400028182A12281C2A16A60A482B2808AC00AC
:10055000A60A482B2C082806031DB02AA601482B02
:100560002818AA11281CAA15A60A482B2808AC008E
:10057000A60A482B2C082806031DC02AA601482BD2
:1005800028182A11281C2A15A60A482B2808AC006E
:10059000A60A482B2C082806031DD02AA601482BA2
:1005A0002818AA10281CAA14A60A482B2808AC0050
:1005B000A60A482B2C082806031DE02AA601482B72
:1005C00028182A10281C2A14A60A482B2808AC0030
:1005D000A60A482B2C082806031DF02AA601482B42
:1005E0002818A912281CA916A60A482B2808AC000E
:1005F000A60A482B2C082806031D002BA601482B11
:1006000028182912281C2916A60A482B2808AC00ED
:10061000A60A482B2C082806031D102BA601482BE0
:100620002818A911281CA915A60A482B2808AC00CF
:10063000A60A482B2C082806031D202BA601482BB0
:1006400028182911281C2915A60A482B2808AC00AF
:10065000A60A482B2C082806031D302BA601482B80
:100660002818A910281CA914A60A482B2808AC0091
:10067000A60A482B2C082806031D402BA601482B50
:1006800028182910281C2914A60A482BA601301462
:1006900008002D10AD10871E2D14871FAD14080003
:1006A0002810071B2814080027082602031C5A2BB1
:1006B0002608A70008002E10BD030310BC0CBB0CBD
:1006C000BA0CB90C03182E140800B400B40B662B36
:1006D0000800BA01BB01BC01A030B900B709371C42
:1006E0003A143718BA14351E3A15351ABA15B51D0D
:1006F0003A16B519BA16351D3A173519BA17B51C79
:100700003B14B518BB14351C3B153518BB15B61E6C
:100710003B16B61ABB16361E3B17361ABB17B61D4C
:100720003C14B619BC14361D3C153619BC15B61C44
:100730003C16B618BC16361C3C173618BC172130B0
:10074000BD000800BE01BF010830C0000310C20C8C
:10075000BF0DBE0DC10CBF0DBE0DC00BA62B0800FA
:10076000C300C4010830C5000310C30CC40DC50B81
:10077000B42B44080800C6000000C60BBC2B0800C0
:10078000CD0A4D080F3C0319CD014D08B800F90101
:10079000F8010800CD034D08013E031DD22B0E3099
:1007A000CD00B800F901F80108002908CD00B80013
:1007B000F13E031CDF2B0E30CD024D08D82BF90182
:1007C000F8010800C7002010201CE42BC70BE32B06
:1007D00008004D0AB023CF00D001D101D201D301CE
:1007E000D40170305718D000FF30EB24CF01D00176
:1007F000D1010130EB2408000530C800EE30C900FB
:1008000003104D0DF9008B13E1258B17CA0003145B
:100810004D0DF9008B13E1258B17C9004A08C8005C
:10082000080021304802031D192C49087907462485
:100830002B2C8B130A08CB0048087807DB00031029
:1008400049087907DC000318DB0AE825CC004B08CF
:100850008A004C088B17F90F2E2CF80A0800831613
:1008600003178C18312C8B130C158312031779087E
:100870008D0077088C008316031755308D00AA3041
:100880008D008C148B178312031308008B138316AF
:1008900003178C18492C0C11831203178D00831633
:1008A00003178C130C14831203170C088312031301
:1008B0008B17080000304624D70008005A24571C24
:1008C000632C5710642C57140030F9005708F700B8
:1008D0002F24E923E9230800FC23F901F80111245E
:1008E000CE00CE131124D600D60A1124D800301C15
:1008F000952C07302A02031D802CD523B0016C2CC7
:10090000AA08031D952C203029020319C023213089
:1009100029020319CA23003029020319CD010C3022
:10092000290203195E24B0016C2C2D080319AB2C8D
:10093000E923E92303302D0203195E242D18A32C8B
:10094000AD18A72C6C2CC023E923E9239A2CCA23C9
:10095000E923E9239A2C17304E0204308A00031948
:10096000D82404308A001B304E0208308A00031954
:10097000002804308A003D08003E031DCB2CA01C3B
:10098000CB2CA010571CC62CC0236C2C0730B500F4
:100990003808B6006923D80B772C6C2C590D590DEB
:1009A000591A013AD91A013AD919013AD90008005D
:1009B0001124CF001124D0001124D1001124D20021
:1009C0001124D3001124D4003030DA005608EB246F
:1009D000DA0BE62C0800D500AE3084008001D21B73
:1009E0008009B33084008001521B8009AF3084003D
:1009F0008001D21A8009AB3084008001521A80092C
:100A0000AA3084008001D2198009A23084008001BC
:100A100052198009A33084008001D2188009A730C0
:100A20008400800152188009A63084008001D31B05
:100A30008009A53084008001531B8009A130840007
:100A40008001D31A8009A03084008001531A8009E4
:100A5000CC3084008001CF1B8009C8308400800125
:100A60004F1B8009C93084008001CF1A8009CA3029
:100A7000840080014F1A8009CE3084008001CF1994
:100A80008009CF30840080014F198009C130840073
:100A90008001CF188009BC30840080014F18800984
:100AA000C03084008001D01B8009C43084008001E4
:100AB000501B8009C53084008001D01A8009CD30D8
:100AC00084008001501A80095508E2230800023092
:100AD0002602031C0301CF000030D0000130EB24BC
:100AE0002D080319832DA701A6013D08003E031D13
:100AF000702D2D08D000CF010130EB24B5010C3052
:100B0000B6006923702D301C672DB001F030CF0086
:100B1000D0017F30EB24CF01D0013F30EB24F03007
:100B2000CF00D0017F30EB242908CF002A08D00065
:100B3000FF30EB24FF30EB24A701A601672D8501D0
:100B40008101CD01BD01AB01AA01A901AC01A60142
:100B5000A701B001A101A201A301AD0183160313F6
:100B600071308F04831603178801890183160313DC
:100B70008230810083160313E03087008312031351
:100B8000AD011D30D9008B168B17FF30CF00D00080
:100B9000D100FF30EB24FF30EB24CF01D001D10195
:100BA000FF30EB24FF30EB24FF30EB245A242D08D8
:100BB000D000FF30EB24FF30EB242D1C6C2C5E2486
:100BC000672D48088A007908490703188A0A8200B5
:100BD0000A08CB005B088A005C0882000834B7343E
:100BE00009340234093417340934623409347D3449
:100BF0000934E0340934F5340A3428340A343D34F5
:100C00000A3452340A3479340B3430340B3481349E
:080C10000B34D2340B34F9342B
:10100000D50004308A001124CF001124D00011240F
:10101000D1001124D2001124D3001124D4000830AF
:101020008A006430BF00AE308400D21BAF20D21FD4
:10103000B320B3308400521BAF20521FB320AF3017
:101040008400D21AAF20D21EB320AB308400521AD3
:10105000AF20521EB320AA308400D219AF20D21D77
:10106000B320A23084005219AF20521DB320A33008
:101070008400D218AF20D21CB320A73084005218AD
:10108000AF20521CB320A6308400D31BAF20D31F47
:10109000B320A5308400531BAF20531FB320A130D1
:1010A0008400D31AAF20D31EB320A0308400531A7B
:1010B000AF20531EB320CC308400CF1BAF20CF1FF6
:1010C000B320C83084004F1BAF204F1FB320C9305E
:1010D0008400CF1AAF20CF1EB320CA3084004F1A2D
:1010E000AF204F1EB320CE308400CF19AF20CF1DCC
:1010F000B320CF3084004F19AF204F1DB320C13033
:101100008400CF18AF20CF1CB320BC3084004F1810
:10111000AF204F1CB320C0308400D01BAF20D01FA5
:10112000B320C4308400501BAF20501FB320C53003
:101130008400D01AAF20D01EB320CD308400501AC6
:10114000AF20501EB320550803308A00E223083038
:101150008A00BF0B1328831304308A00BB2C800A3B
:101160000319800908008008031D80030800173454
:1011700010340C34803400340034803400340034B3
:10118000403400340034403400340034203400341F
:10119000003420340034003410340034003410346F
:1011A000003400340834003400340834003400348F
:1011B0000434003400340434003400340234003485
:1011C000003402340034003401340034003401347B
:1011D000003400340034803400340034803400346F
:1011E00000344034003400344034003400342034BF
:1011F000003400342034003400341034003400341F
:1012000010340034173410340334FF34FF34FF3407
:10121000FF34FF34FF34FF34F0340034FF34F03453
:10122000003400340F34FF3400340F34FF341734EB
:1012300003340C34803410340034803410340034DF
:1012400040342034003440342034003420344034DE
:1012500000342034403400341034803400341034EE
:10126000803400340934003400340934003400344C
:101270000634003400340634003400348034103432
:10128000003480341034003440342034003440348E
:1012900020340034203440340034203440340034CE
:1012A0001034803400341034803400340934003475
:1012B0000034093400340034063400340034063479
:1012C00000340034173410340434FC340F34C03488
:1012D000003400340034003400340034FC340F3463
:1012E000C0340334F0343F3400340034003400346C
:1012F000003400340334F0343F341B3410341034E1
:10130000FF34FF34FF34FF34FF34FF34FF34FF3445
:10131000FF34FF34FF34FF34FF34FF34FF34FF3435
:10132000FF34FF34FF34FF34FF34FF34FF34FF3425
:10133000003400340034003400340034003400340D
:1013400000340034003400340034003400340034FD
:1013500000340034003400340034003400340034ED
:10136000FF34F0340034FF34F0340034FF34F03410
:101370000034FF34F0340034FF34F0340034FF34F0
:10138000F0340034FF34F0340034FF34F0340034EF
:1013900000340034003400340034003400340034AD
:1013A000003400340034003400340034003400349D
:1013B000003400340034003400340034003400348D
:1013C000173403340334DB346D34B634DB346D341A
:1013D000B6346D34B634DB346D34B634DB34B63405
:1013E000DB346D34B634DB346D34173402340834F6
:1013F00080341034003480341034003440342034CD
:101400000034403420340034A03450340034A0344C
:10141000503400345034A03400345034A0340034FC
:1014200029344034003429344034003416348034B4
:101430000034163480340034093400340034093464
:1014400000340034063400340034063400340034F0
:10145000173403340334DB3460340034DB34603459
:1014600000346D34B03400346D34B0340034B634EC
:10147000D03400346D34B0340034173403340334C2
:1014800092344034003492344034003449342034AF
:10149000003449342034003424349034003424346B
:1014A00090340034173403340634C33401348634A2
:1014B000C3340134863461348034C33461348034BD
:1014C000C3343034C83461343034C83461341834EF
:1014D0006C34303418346C3430340C3436341834C2
:1014E0000C3436341834863413340C3486341334C4
:1014F0000C341B3403341E34803400340134003483
:1015000000340034C0340034033400340034003478
:10151000E03400340734003400340034F034003454
:101520000F34003400340034783400341E34003476
:10153000003400343C3400343C3400340034003493
:101540001E34003478340034003400340F34003456
:10155000F03400340034003407348134E034003493
:10156000003400340334C334C03400340034003455
:101570000134E73480340034003400340034FF3464
:10158000003400340034003400347E34003400343D
:101590000034003400343C3400340034003400346F
:1015A0000034183400340034003400340034003483
:1015B0000034803400340134003400340034C0344A
:1015C00000340334003400340034E0340034073491
:1015D000003400340034F03400340F34003400346C
:1015E0000034783400341E340034003400343C3489
:1015F00000343C340034003400341E340034783479
:101600000034003400340F340034F034003400343B
:10161000003407348134E0340034003400340334BF
:10162000C334C0340134003400340134E73480342E
:101630000034003400340034FF340034003400340B
:10164000003400347E34003400340034003400347C
:101650003C34003400340034003400341834003496
:101660001B3403340D34803410340034803410348F
:101670000034C03430340034C03430340034E0340A
:1016800070340034E03470340034F034F03400341A
:10169000F034F03400347934E03400347934E03418
:1016A00000343F34C03400343D34C03400341F347F
:1016B000803400341F34803400340F34003400345C
:1016C0000F3400340034063400340034063400345F
:1016D000003400340034003400340034003400346A
:1016E000003400340034003400340034003400345A
:1016F000003400340034003400340034003400344A
:1017000000341B3403340D34063400340034063402
:10171000003400340F34003400340F34003400340B
:101720001F34803400341F34803400343F34C034DC
:1017300000343D34C03400347934E034003479343A
:10174000E0340034F034F0340034F034F034003459
:10175000E03470340034E03470340034C034303459
:101760000034C034303400348034103400348034D9
:1017700010340034003400340034003400340034B9
:1017800000340034003400340034003400340034B9
:1017900000340034003400340034003400340034A9
:1017A00000340034173403340634803410340034E9
:1017B0008034103400342034403400342034403439
:1017C0000034093400340034093400340034403427
:1017D0002034003440342034003410348034003459
:1017E00010348034003406340034003406340034BD
:1017F0000034173401342134C03430340034C03460
:101800003034003400340034003400340034003408
:10181000C03430340034C034303400340034003448
:10182000003400340034003400340C340334003409
:101830000C340334003400340034003400340034F9
:1018400000340C34033400340C34033400340034DA
:1018500000340034003400340034003400340034E8
:1018600000340034003400340034003400340034D8
:101870000034003400340034003400343034C034D8
:1018800000343034C03400340034003400340034C8
:10189000003400343034C03400343034C0340034C8
:1018A0000034003400340034003400340034033495
:1018B0000C34003403340C3400340034003400346D
:1018C00000340034003403340C34003403340C345A
:1018D0000034003400340034003400340034003468
:1018E0000034003400340034003400340034003458
:1018F0000034003400340034003400340034003448
:101900000F34003400340F34003400340034003419
:1019100000340034003400340F34003400340F3409
:101920000034003400340034003400340034003417
:1019300000340034F03400340034F0340034003427
:10194000003400340034003400340034F034003407
:101950000034F034003400340034003400340034F7
:1019600000340034003400340034003400340034D7
:1019700000340034003400340034003400340034C7
:0419800000340034FB
:02400E00C428C4
:02401000FF3E71
:02420000FF3489
:00000001FF
